:100000000C942A000C9445000C9445000C94450077
:100010000C9445000C9445000C9445000C9445004C
:100020000C9445000C9445000C9445000C9445003C
:100030000C9445000C9445000C9445000C9445002C
:100040000C9445000C9445000C9445000C9445001C
:100050000C94450011241FBECFE5D8E0DEBFCDBF14
:1000600010E0A0E6B0E0ECE5F1E002C005900D92F2
:10007000A036B107D9F710E0A0E6B0E001C01D92AC
:10008000A036B107E1F70C948C000C940000CF93DC
:10009000DF93CDB7DEB7809153008966809353001C
:1000A00080913700886080933700DF91CF91089569
:1000B000CF93DF93CDB7DEB721970FB6F894DEBFAD
:1000C0000FBECDBF8983898180935C0021960FB6D6
:1000D000F894DEBF0FBECDBFDF91CF910895CF93CF
:1000E000DF93CDB7DEB722970FB6F894DEBF0FBE11
:1000F000CDBF80E89CE09A83898389819A810197AA
:10010000F1F79A83898322960FB6F894DEBF0FBE6B
:10011000CDBFDF91CF910895CEE5D8E0DEBFCDBF52
:1001200019820E944700198289818F3F49F0898195
:100130000E9458000E946F0089818F5F8983F4CFED
:100140008FEF89838981882371F389810E94580008
:0C0150000E946F00898181508983F4CFE8
:00000001FF
